:020000040000FA
:1000000036288207003400340034003400344C3485
:100010004B34403400349834963480340034E43423
:10002000E134C034013431342D34003401347D34B2
:10003000783440340134C934C33480340234163443
:100040000E34C034023462345A3400340234AE34D4
:10005000A53440340234FA34F03480340334473465
:100060003B34C03403349334873400348B0183161B
:100070008113FB308500860183120511BA20FD2013
:10008000051A4328F221890185230808A300852346
:100090000808A40085230808A50085230808A600F1
:1000A000852308088C00852308088D00852308080F
:1000B0008E00852308088F00DD220B238C22C322AB
:1000C000C3220508B30003303305B200B00140304D
:1000D000AF00B401B6019021B319702890206B28AD
:1000E0009D019C019B0101309A00331A8128E83060
:1000F0009A0003309B00812803109A0D9B0D9C0DE4
:100100009D0DAF0DB00D031C7C28B41889287D21EE
:100110008B2840215821DD220B238C22C3226B28FF
:10012000B4189C280430B602CF303607031C9A2836
:100130003030B600A820A3280430B607CF303607E9
:100140000318B601A820DD220B238C22C32208004D
:10015000360801208F00B60A360801208E00B60A44
:10016000360801208D00B60A360801208C000330C5
:10017000B602080095230330860006169523061262
:1001800003308600061698230612033086000616F2
:10019000982306120230860006169B23061228308A
:1001A00056230830562301305623063056230C3090
:1001B00056230800C030562320305A2320305A23BB
:1001C00020305A2320305A2320305A2320305A23FB
:1001D00020305A2320305A2320305A2320305A23EB
:1001E00020305A2320305A2320305A2320305A23DB
:1001F00020305A2320305A230800813056235630AD
:100200005A2346305A234F305A2320305A23443041
:100210005A2344305A2353305A2320305A23413032
:100220005A2344305A2339305A2338305A23353030
:100230005A2331305A238A23C030562346305A235A
:1002400052305A2345305A2351305A2355305A23BD
:1002500045305A234E305A2343305A2345305A23CF
:1002600020305A2353305A234F305A2352305A23C6
:1002700054305A2349305A2345305A238A230800E0
:100280001A088C07031C49298D0F49298E0F49290B
:100290008F0A1B088D07031C50298E0F50298F0AC7
:1002A0001C088E07031C55298F0A1D088F0708009C
:1002B000FC300F070318742903300F02031C7C293C
:1002C0006C300E070318742993300E02031C7C292E
:1002D00078300D070318742987300D02031C7C2920
:1002E00000300C02031C7C2900308C0087308D000C
:1002F00093308E0003308F0008009A099B099C09F7
:100300009D099A0F88299B0F88299C0F88299D0A8F
:1003100040218F1F8F298C018D018E018F010800D4
:10032000B0014030AF00B921B01B9A290830AF07A7
:100330000318B00A0508B30003303305B1003206D4
:10034000031993290310B20D3108B206320802399D
:10035000B50034060319B1293508B4003108B200DC
:100360009329B401B21CB6290230B4003108B2009E
:100370000800051EBE298519C729C3298519C52965
:100380003818C929DC293814F1293810F129B801A5
:10039000F1291030B900051AD2299223B90BCB29C3
:1003A0007D22F1299D010F309C0042309B0040309E
:1003B0009A0040215821ED291030B9008519E5290E
:1003C0009223B90BDE297D22F1299D010F309C007B
:1003D00042309B0040309A007D21DD220B238C228D
:1003E000C322080080308C0096308D0098308E003B
:1003F00000308F00890185230808A30085230808A1
:10040000A40085230808A50085230808A600DD228E
:100410000B23C030AB0056232030AB005A234330AF
:10042000AB005A234130AB005A234C30AB005A2367
:100430004930AB005A234230AB005A235230AB0054
:100440005A234130AB005A235430AB005A23493071
:10045000AB005A234F30AB005A234E30AB005A2327
:100460002E30AB005A232E30AB005A232E30AB0077
:100470005A232030AB005A238C22C32290219D01A5
:100480009C019B0110309A003319482A80309A0051
:100490000000B418562A9A099B099C099D099A0FD5
:1004A000562A9B0F562A9C0F562A9D0A1A08A30704
:1004B000031C5F2AA40F5F2AA50F5F2AA60A1B0848
:1004C000A407031C662AA50F662AA60A1C08A5070E
:1004D000031C6B2AA60A1D08A607051E3C2A8901D3
:1004E00023088800782324088800782325088800BA
:1004F00078232608880078230800043089000C0837
:10050000880078230D08880078230E088800782357
:100510000F0888007823080095019601970198013B
:1005200099012030A0002308A7002408A80025086E
:10053000A9002608AA000310271CB52A0C08960754
:10054000031CA72A970FA72A980FA72A990A0D0814
:100550009707031CAE2A980FAE2A990A0E0898072F
:10056000031CB32A990A0F089907990C980C970C49
:10057000960C950CAA0CA90CA80CA70CA00B9B2AF6
:10058000013099000800153084000008A2000830EE
:10059000A100A20C031CD02A861506150611D32A29
:1005A000861106150611A10BC92A840A1A30040205
:1005B000031CC52A86178613080020309E00900170
:1005C000910192019301940103108C0D8D0D8E0DFC
:1005D0008F0D03180C14900D910D920D930D940D29
:1005E0009E03031DF42A0800103084000023840AAF
:1005F0000023840A0023840A0023840A0023E42AB7
:10060000033000079F009F198000303000079F00D3
:100610009F1B800008008030562320305A23130E81
:100620000F39303E5A2313080F39303E5A232C30ED
:100630005A23120E0F39303E5A2312080F39303E1A
:100640005A23110E0F39303E5A232E305A231108E7
:100650000F39303E5A23100E0F39303E5A231008FE
:100660000F39303E5A2320305A234D305A23483018
:100670005A237A305A2320305A23080086018316E1
:1006800008308600831206138616FF30AD0006166A
:100690000608AC0006120000000006160000061254
:1006A000AD030319552BAC19472B0800AB00B7015C
:1006B00006135D2BAB00371406173E238601831605
:1006C0000030860083128612061337180617F030A2
:1006D00086052B0E0F398604061600000612F03030
:1006E00086052B080F39860406160000061208003E
:1006F0008316081555308900AA3089008814881897
:100700007F2B08118312890A0800831608148312AC
:10071000890A08008F238F238F238F2308009223B9
:1007200092230800FF30AD00A02B8030AD00A02B3D
:100730004030AD00A02B2030AD00A02B1030AD001C
:0E074000FF30AE00AE0BA22BAD0BA02B0800BD
:084000007F007F007F007F00BC
:02400E00F13F80
:10420000DE006500DC0017008000C300C90001006B
:10421000000000000000000000000000000000009E
:10422000000000000000000000000000000000008E
:10423000000000000000000000000000000000007E
:10424000000000000000000000000000000000006E
:10425000000000000000000000000000000000005E
:10426000000000000000000000000000000000004E
:10427000000000000000000000000000000000003E
:00000001FF
